:0200000480007A
:100000006F000005732F2034930F80006308FF03F7
:10001000930F90006304FF03930FB0006300FF038E
:10002000130F000063040F0067000F00732F2034CC
:1000300063540F006F00400093E19153171F0000BD
:1000400023223FFC171F000023200FFC6FF01FFF2F
:100050009300000013010000930100001302000050
:100060009302000013030000930300001304000038
:100070009304000013050000930500001306000020
:100080009306000013070000930700001308000008
:10009000930800001309000093090000130A0000F0
:1000A000930A0000130B0000930B0000130C0000D8
:1000B000930C0000130D0000930D0000130E0000C0
:1000C000930E0000130F0000930F0000732540F102
:1000D0006310050097020000938202017390523072
:1000E000735044749702000093820201739052305F
:1000F00073500018970200009382020273905230EE
:10010000B70200809382F2FF7390023B9302F001EA
:100110007390023A7350403097020000938242017C
:100120007390523073502030735030309301000080
:1001300097020000938242ED739052301305100035
:100140001315F501634C05000F00F00F930110002B
:100150009308D0051305000073000000930200000F
:10016000638A020073905210B7B20000938292101B
:100170007390223073500030970200009382420146
:1001800073901234732540F17300203093012000E6
:100190009307F00F972000009380C0E603D700007C
:1001A0009303F00F6310772A93013000B707010023
:1001B000938707F0972000009380C0E403D72000C6
:1001C000B7030100938303F0631E77269301400079
:1001D000B7170000938707FF97200000938080E205
:1001E00003D74000B7130000938303FF631C7724F9
:1001F00093015000B7F700009387F70097200000A5
:10020000938040E003D76000B7F300009383F300CE
:10021000631A7722930160009307F00F9720000084
:100220009380A0DE03D7A0FF9303F00F631C772019
:1002300093017000B7070100938707F09720000033
:100240009380A0DC03D7C0FFB7030100938303F0C2
:10025000631A771E93018000B7170000938707FF8A
:1002600097200000938060DA03D7E0FFB713000007
:10027000938303FF6318771C93019000B7F7000086
:100280009387F70097200000938020D803D70000C1
:10029000B7F300009383F3006316771A9301A0006D
:1002A00097200000938000D6938000FE83D2000246
:1002B0009303F00F639872189301B0009720000029
:1002C000938040D49380B0FF83D27000B7030100C5
:1002D000938303F0639872169301C0001302000029
:1002E00097200000938020D203D72000130307003B
:1002F000B7130000938303FF6316731413021200F5
:1003000093022000E31E52FC9301D0001302000070
:1003100097200000938040CF03D7200013000000F7
:1003200013030700B7F300009383F300631C7310FB
:100330001302120093022000E31C52FC9301E00020
:1003400013020000972000009380C0CB03D7200049
:10035000130000001300000013030700B70301009F
:10036000938303F06310730E1302120093022000B4
:10037000E31A52FC9301F0001302000097200000E2
:10038000938060C803D72000B7130000938303FF56
:10039000631A770A1302120093022000E31052FE40
:1003A0009301000113020000972000009380C0C554
:1003B0001300000003D72000B7F300009383F3007D
:1003C000631277081302120093022000E31E52FC0E
:1003D000930110011302000097200000938080C257
:1003E000130000001300000003D72000B703010032
:1003F000938303F063187704130212009302200022
:10040000E31C52FC9301200197220000938282BFDB
:1004100003D1020013012000930320006314710232
:1004200093013001972200009382C2BD03D10200E4
:1004300013000000130120009303200063147100D7
:10044000631030020F00F00F6380010093911100E0
:1004500093E111009308D00513850100730000009B
:100460000F00F00F930110009308D0051305000052
:0C04700073000000731000C000000000CA
:1010000000000000000000000000000000000000E0
:1010100000000000000000000000000000000000D0
:1010200000000000000000000000000000000000C0
:1010300000000000000000000000000000000000B0
:081040000000000000000000A8
:10200000FF0000FFF00F0FF00000000000000000D4
:040000058000000077
:00000001FF
